:02000000F028E6
:100008001029A601A500BA172730A400103018201F
:100018000330A400E8301820A40164301820A4019B
:100028000A30182025082328A3002608A20025083E
:10003800A100B9202108031DBA13BA1B0800303EDD
:10004800A7003E0884000930A80003103020A70C40
:10005800A80B2A28031430288413BA1D3F28000847
:100068003C043A1D3C068000841700083C04031C2D
:100078003C0680004A2800083C04031C3C063A1948
:100088003C06800084173C0980054A283A0D063949
:10009800A1005320A200A10A532000007E280030AE
:1000A8008A00210882070134993403343934003432
:1000B80060340C34FD3483169B001C141A08EB289A
:1000C80083169A001C1555309D00AA309D009C147B
:1000D8009C186C281C11EB28A401A300FF30A3076F
:1000E800031CA407031CEB280330A200E6307E2083
:1000F8007228A201FC3EA100A209031C8928FF3036
:100108000000A10703188428A1076400A20F832810
:100118000800A201A401A30002309E28A300033016
:100128009E28A30001309E28A30006309E28A30025
:1001380004309E28A90024082202031DA5282308AC
:100148002102043003180130031902302905031D68
:10015800FF30EB280038031DFF300405031DFF3076
:10016800EB280404031DFF30EB28A601A50110307D
:10017800A700220DA50DA60D2308A5022408031C1F
:10018800240FA6020318CF282308A507240803185C
:10019800240FA6070310A10DA20DA70BBD28210847
:1001A800EB281030A900A201A101A80CA70C031C80
:1001B800E3282308A10724080318240FA207A20C88
:1001C800A10CA60CA50CA90BD9282508EB2883138C
:1001D8000313831264000800831681138312073007
:1001E8009F0083168F3086000430850083123130DB
:1001F8009000C0308B00831601308C008312DC30F5
:10020800C3000B30C2000A30C400C5015830D20008
:100218000230D300E0018B29A000030E8301C00047
:100228000A08BB0043088E0042088F00C10A0C1060
:100238003B088A00400E8300A00E200E09006400CF
:100248000A304102031C6F2983168C01831241086E
:10025800A100A2010A30A300A401B920B30022081A
:10026800B4003308E4074108A100A2010A30A30042
:10027800A401B920B3002208B4003308DE0734080B
:100288000318013EDF074108A100A2010A30A300BC
:10029800A401B9202508C100831601308C0008305C
:1002A800831285068316851164003C30831264022C
:1002B800031C6F293C30E402E20A64003C3062020D
:1002C800031C6F29E201E10A64000D306102031C7E
:1002D8006F290130E1000800E10A64000D30610275
:1002E800031C78290130E1000800E20A64003C3070
:1002F8006202031C8829E201E10A64000D306102F0
:10030800031C88290130E1000800E4010800F124F9
:10031800232164000519AB29DF2285118316851175
:100328008312E6240530BE000230BC000630BA0055
:10033800610805203A302420620805203A3024203C
:10034800640805200330A400E83071208C29F721C7
:10035800EC2264000618B1294A2B4108A10000309C
:100368008D20B3006408A10000308D20B50033084B
:1003780084003508AE20B500B6006208A100003040
:100388008D20B7003508360484003708AE20B70042
:10039800B8006400370838040319F6296400E31824
:1003A800F629E6240530BE000230BC000630BA004B
:1003B80054302420693024206D30242065302420D6
:1003C8002030242069302420733024202030242039
:1003D800610805203A302420620805203A3024209C
:1003E800640805208C296108A700A8015608A30005
:1003F8005708A400D520B3002608B4003308A1008C
:100408003408A2000A30A300A401B920C8002208B9
:10041800C9006208A700A8015808A3005908A40049
:10042800D520B3002608B4003308A1003408A20080
:100438000A30A300A401B920CA002208CB0064082E
:10044800A700A8015A08A3005B08A400D520B300A0
:100458002608B4003308A1003408A2000A30A3001B
:10046800A401B920CC002208CD006400861B582ABC
:100478004108A700A8015A08A3005B08A400D520DA
:10048800B3002608B4003308A1003408A200643081
:10049800A300A401B920B3002208B4003308CC0794
:1004A80034080318013ECD07003006180130A100BA
:1004B80000308D20B300003063190130A1000130F5
:1004C8008D20B500330884003508B520B500B60086
:1004D8006400350836040319942AC801C901CA0101
:1004E800CB01CC01CD0164006008003C031D812ACA
:1004F8004E08C8004F08C900942A64006008013CEF
:10050800031D8B2A5008CA005108CB00942A6400A6
:100518006008023C031D942A5408CC005508CD00FD
:10052800D222DC01DD015C08A1005D08A2005308AD
:10053800A40052089520031DD12A5C08A1005D087B
:10054800A2004908A40048089B20031DAF2A0612F0
:100558008316061283125C08A1005D08A2004B08EE
:10056800A4004A089B20031DBD2A86128316861202
:1005780083125C08A1005D08A2004D08A4004C0885
:100588009B20031DCB2A0613831606138312013002
:100598007D20DC0A0319DD0F972A0800061683164A
:1005A800061283128616831686128312061783167E
:1005B8000613831208000612831606128312861287
:1005C80083168612831206138316061383120800F5
:1005D800631064008618F22A7021631464000619F7
:1005E800F72A7921631464008619FC2A8921631487
:1005F8006400631C492B0130C600C7014608A100EE
:100608004708A2004508A40044089520031D112BA3
:10061800F721C60A0319C70F022B6400E318492BF8
:10062800E6240530BE000230BC000630BA00553062
:100638002420703024206430242061302420743039
:100648002420653024206430242020302420743075
:100658002420693024206D30242065302420203067
:10066800242069302420733024202030242061087D
:1006780005203A302420620805203A3024206408F6
:1006880005203A3024204108052008006310640042
:10069800061C512BAD246A248C29640086185F2B14
:1006A800E00A6008A100A2010330A300A401B92058
:1006B8002508E000631464000619872B64006008AD
:1006C800003C031D6E2B0130CE020030031C013E9E
:1006D800CF02852B64006008013C031D7A2B013092
:1006E800D0020030031C013ED102852B6400600853
:1006F800023C031D852B0130D4020030031C013E4F
:10070800D5021B24631464008619A62B64006008B4
:10071800003C031D932BCE0A0319CF0AA42B6400B7
:100728006008013C031D9C2BD00A0319D10AA42B95
:1007380064006008023C031DA42BD40A0319D50ADF
:100748001B2463146400631CE32BE62364008618EF
:10075800CB2B0130C600C7014408A7004508A800F4
:100768000230A300A401D520B3002608B40046082F
:10077800A1004708A2003408A40033089520031DEF
:10078800CA2BF721C60A0319C70FB02BE22B013079
:10079800C600C7010310450CB400440CB30046085A
:1007A800A1004708A2003408A40033089520031DBF
:1007B800E22BF721C60A0319C70FCE2BE42BF7212A
:1007C80023214A2B6400E3181A2C0530BE0002309E
:1007D800BC000630BA0068302420203024204F089E
:1007E800A6004E08062020302420203024206D301A
:1007F8002420203024205108A6005008062020304C
:100808002420203024207330242020302420550830
:10081800A600540806206D3024206F302420643050
:1008280024206530242060080520E62408004E08AE
:10083800A1004F08A200A40101309220031D272C1B
:100848000130CE00CF015008A1005108A200A40138
:1008580001309220031D332C0130D000D1015408FF
:10086800A1005508A200A40101309220031D3F2CCD
:100878000130D400D5014E08A1004F08A20053084A
:10088800A40052089820031D4D2C5208CE0053088E
:10089800CF005008A1005108A2005308A400520834
:1008A8009820031D5B2C5208D0005308D10054082F
:1008B800A1005508A2005308A40052089820031D5F
:1008C800692C5208D4005308D50008004E08A70028
:1008D8004F08A8000A30A300A401D520B3002608B9
:1008E800B4003308A1003408A2000C30A300A4010E
:1008F800B920D6002208D7005008A7005108A80040
:100908000A30A300A401D520B3002608B400330898
:10091800A1003408A2003C30A300A401B920D800EB
:100928002208D9005408A7005508A8000A30A300D7
:10093800A401D520B3002608B4003308A100340868
:10094800A2003C30A300A401B920DA002208DB0091
:100958000800831601309B0083124F086420831619
:1009680002309B0083124E086420831603309B00DC
:10097800831251086420831604309B0083125008A8
:100988006420831605309B00831255086420831663
:1009980006309B00831254086420080001305F2051
:1009A800CF0002305F20CE0003305F20D10004303A
:1009B8005F20D00005305F20D50006305F20D400CE
:1009C8001B2408000530BE000230BC000630BA0007
:1009D8000A3024200D30242008006315DF228515F5
:1009E800831685118312E624E6240530BE00023002
:1009F800BC000630BA00413024206C30242061301D
:100A080024206E30242027302420733024202030E6
:100A18002420453024206C30242065302420633085
:100A2800242074302420723024206F3024206E302B
:100A380024206930242063302420203024205030A2
:100A48002420723024206F3024206A30242065301E
:100A58002420633024207430242073302420203054
:100A68002420493024206E302420633024202E3066
:100A78002420E6240530BE000230BC000630BA004F
:100A88004D302420753024206C30242074302420EC
:100A9800693024206D3024206530242074302420CF
:100AA8006530242072302420203024204330242034
:100AB8006C3024206F302420633024206B302420B5
:100AC800E6240530BE000230BC000630BA002D30E6
:100AD80024202D3024202D3024202D3024202D308A
:100AE80024202D3024202D3024202D3024202D307A
:100AF80024202D3024202D3024202D3024202D306A
:100B080024202D3024202D3024202D3024202D3059
:100B180024202D3024202D3024202D3024202D3049
:100B280024202D3024202D3024202D3024202D3039
:100B380024202D302420E6240530BE000230BC00DD
:100B48000630BA0048302420203024203D302420AC
:100B5800203024204F08A6004E0806202C302420E0
:100B6800203024204D302420203024203D302420E3
:100B7800203024205108A600500806202C302420BC
:100B88002030242053302420203024203D302420BD
:100B9800203024205508A60054080620E624E62420
:100BA800E314D2246A240C30E100E201E401C1011B
:100BB800DE01DF01E0010130E50064006530650217
:100BC8000318E92DF721E50FE12D0130E000013090
:100BD800E5006400653065020318F52DF721E50F7F
:100BE800ED2D0230E0000130E5006400653065025B
:100BF8000318012EF721E50FF92DE001E624053051
:100C0800BE000230BC000630BA00533024207430D5
:100C18002420613024207230242074302420753040
:100C280024207030242020302420633024206F308A
:100C380024206D302420703024206C30242065302E
:100C4800242074302420653024202E302420E624EB
:040C5800631108001C
:02400E00063F6B
:0C42020001002C0001002C0001002C0029
:00000001FF
